:100000000C9446000C9465000C9465000C946500FB
:100010000C9465000C9465000C9465000C946500CC
:100020000C9465000C9465000C9465000C946500BC
:100030000C9465000C9465000C9465000C946500AC
:100040000C9465000C9465000C9465000C9465009C
:100050000C9465000C9465000C9465000C9465008C
:100060000C9465000C9465000C9465000C9465007C
:100070000C9465000C9465000C9465000C9465006C
:100080000C9465000C9465000C94650011241FBE4F
:10009000CFEFD0E1DEBFCDBF11E0A0E0B1E0E8E6F8
:1000A000F1E000E00BBF02C007900D92A030B10755
:1000B000D9F711E0A0E0B1E001C01D92A030B10776
:1000C000E1F70E9467000C94B3000C940000CF93FA
:1000D000DF93CDB7DEB722970FB6F894DEBF0FBE21
:1000E000CDBFE8E3F0E080E88083E7E3F0E080E87C
:1000F0008083E2E3F0E01082E1E3F0E0108200C0F0
:10010000E0E3F0E08081992784709070009719F502
:10011000E6E3F0E08081882344F4A8E3B0E0E8E37C
:10012000F0E080818F778C9307C0A8E3B0E0E8E32C
:10013000F0E0808180688C9380E395E79A838983DF
:1001400005C089819A8101979A83898389819A81DF
:100150000097B9F7D5CFA8E3B0E0E8E3F0E08081FD
:0801600080688C93CDCFFFCF26
:00000001FF
